:020000040800F2
:1000000000800120498D0008098700080B8700083F
:100010000D8700080F870008118700080000000006
:10002000000000000000000000000000138700082E
:1000300015870008000000001787000819870008CE
:10004000998D0008998D0008998D0008998D0008F8
:10005000998D0008998D0008998D0008998D0008E8
:10006000998D0008998D0008998D0008998D0008D8
:10007000998D0008998D0008998D0008998D0008C8
:1000800021870008998D0008998D00080000000064
:10009000000000000000000000000000998D000832
:1000A000998D0008998D0008998D0008998D000898
:1000B00031870008998D0008998D0008998D0008F6
:1000C000998D0008998D0008998D0008998D000878
:1000D000998D000841870008518700080000000042
:1000E000998D0008998D0008998D00080000000086
:1000F000000000000000000000000000998D0008D2
:1001000000000000998D0008998D0008998D000865
:1001100000000000000000000000000000000000DF
:10012000998D0008998D0008998D0008998D000817
:10013000998D000800000000000000000000000091
:10014000000000000000000000000000998D000881
:10015000998D0008998D000861870008998D000825
:10016000998D0008998D0008000000000000000033
:10017000000000000000000000000000000000007F
:1001800000000000998D0008000000000000000041
:04019000998D00083D
:1001A00010B5054C237833B9044B13B10448AFF3B1
:1001B00000800123237010BDE4090020000000002E
:1001C000DCD3000808B5034B1BB103490348AFF368
:1001D000008008BD00000000E8090020DCD3000812
:1001E000034613F8012B002AFBD1181A0138704777
:1001F00001F0FF01102A2BDB10F0070F08D010F8D8
:10020000013B013A8B422DD010F0070F42B3F6D1DB
:10021000F0B441EA012141EA014122F007047FF0F4
:1002200000070023F0E80256083C85EA010586EA4B
:10023000010685FA47F5A3FA87F586FA47F6A5FA87
:1002400087F68EB9EED1F0BC01F0FF0102F0070293
:1002500032B110F8013B013A83EA010313B1F8D13E
:100260000020704701387047002D06BF354603381F
:10027000073815F0010F07D1013015F4807F02BF58
:10028000013015F4C03F0130F0BC0138704700BFA9
:1002900081F0004102E000BF83F0004330B54FEA37
:1002A00041044FEA430594EA050F08BF90EA020FA4
:1002B0001FBF54EA000C55EA020C7FEA645C7FEA37
:1002C000655C00F0E2804FEA5454D4EB5555B8BF5A
:1002D0006D420CDD2C4480EA020281EA030382EACB
:1002E000000083EA010180EA020281EA0303362D5D
:1002F00088BF30BD11F0004F4FEA01314FF4801C30
:100300004CEA113102D0404261EB410113F0004F41
:100310004FEA03334CEA133302D0524263EB4303F8
:1003200094EA050F00F0A780A4F10104D5F1200E96
:100330000DDB02FA0EFC22FA05F2801841F10001F1
:1003400003FA0EF2801843FA05F359410EE0A5F1C5
:1003500020050EF1200E012A03FA0EFC28BF4CF0F6
:10036000020C43FA05F3C01851EBE37101F00045AC
:1003700007D54FF0000EDCF1000C7EEB00006EEBB9
:100380000101B1F5801F1BD3B1F5001F0CD3490843
:100390005FEA30004FEA3C0C04F101044FEA44529A
:1003A00012F5800F80F09A80BCF1004F08BF5FEA21
:1003B000500C50F1000041EB045141EA050130BD01
:1003C0005FEA4C0C404141EB010111F4801FA4F1A4
:1003D0000104E9D191F0000F04BF01460020B1FAF9
:1003E00081F308BF2033A3F10B03B3F120020CDA31
:1003F0000C3208DD02F1140CC2F10C0201FA0CF00F
:1004000021FA02F10CE002F11402D8BFC2F1200C73
:1004100001FA02F120FA0CFCDCBF41EA0C01904029
:10042000E41AA2BF01EB0451294330BD6FEA040472
:100430001F3C1CDA0C340EDC04F11404C4F120025D
:1004400020FA04F001FA02F340EA030021FA04F36F
:1004500045EA030130BDC4F10C04C4F1200220FAC6
:1004600002F001FA04F340EA0300294630BD21FA04
:1004700004F0294630BD94F0000F83F4801306BFCA
:1004800081F480110134013D4EE77FEA645C18BFBE
:100490007FEA655C29D094EA050F08BF90EA020F55
:1004A00005D054EA000C04BF1946104630BD91EA4D
:1004B000030F1EBF0021002030BD5FEA545C05D150
:1004C0004000494128BF41F0004130BD14F580048F
:1004D0003CBF01F5801130BD01F0004545F0FE4103
:1004E00041F470014FF0000030BD7FEA645C1ABF38
:1004F000194610467FEA655C1CBF0B46024650EA6F
:10050000013406BF52EA033591EA030F41F400219A
:1005100030BD00BF90F0000F04BF0021704730B520
:100520004FF4806404F132044FF000054FF00001F5
:1005300050E700BF90F0000F04BF0021704730B5B6
:100540004FF4806404F1320410F0004548BF40428B
:100550004FF000013EE700BF42004FEAE2014FEAE0
:1005600031014FEA02701FBF12F07F4393F07F4FBB
:1005700081F06051704732F07F4208BF704793F0BE
:100580007F4F04BF41F40021704730B54FF46074D1
:1005900001F0004521F000411CE700BF50EA0102D4
:1005A00008BF704730B54FF000050AE050EA01027D
:1005B00008BF704730B511F0004502D5404261EBED
:1005C00041014FF4806404F132045FEA915C3FF42E
:1005D000D8AE4FF003025FEADC0C18BF03325FEACB
:1005E000DC0C18BF033202EBDC02C2F1200300FA7C
:1005F00003FC20FA02F001FA03FE40EA0E0021FAA1
:1006000002F11444BDE600BF70B54FF0FF0C4CF48E
:10061000E06C1CEA11541DBF1CEA135594EA0C0F40
:1006200095EA0C0F00F0DEF82C4481EA030621EA7B
:100630004C5123EA4C5350EA013518BF52EA0335B6
:1006400041F4801143F4801338D0A0FB02CE4FF068
:100650000005E1FB02E506F00042E0FB03E54FF098
:100660000006E1FB03569CF0000F18BF4EF0010E90
:10067000A4F1FF04B6F5007F64F5407404D25FEA8C
:100680004E0E6D4146EB060642EAC62141EA55513F
:100690004FEAC52040EA5E504FEACE2EB4F1FD0C81
:1006A00088BFBCF5E06F1ED8BEF1004F08BF5FEAFF
:1006B000500E50F1000041EB045170BD06F00046B1
:1006C00046EA010140EA020081EA0301B4EB5C045E
:1006D000C2BFD4EB0C0541EA045170BD41F4801156
:1006E0004FF0000E013C00F3AB8014F1360FDEBF7B
:1006F000002001F0004170BDC4F10004203C35DA57
:100700000C341BDC04F11404C4F1200500FA05F3D9
:1007100020FA04F001FA05F240EA020001F000427A
:1007200021F0004110EBD37021FA04F642EB0601F0
:100730005EEA430E08BF20EAD37070BDC4F10C041A
:10074000C4F1200500FA04F320FA05F001FA04F2DE
:1007500040EA020001F0004110EBD37041F10001CA
:100760005EEA430E08BF20EAD37070BDC4F12005D5
:1007700000FA05F24EEA020E20FA04F301FA05F23D
:1007800043EA020321FA04F001F0004121FA04F2E5
:1007900020EA020000EBD3705EEA430E08BF20EAB5
:1007A000D37070BD94F0000F0FD101F000464000EF
:1007B00041EB010111F4801F08BF013CF7D041EA71
:1007C000060195F0000F18BF704703F00046520075
:1007D00043EB030313F4801F08BF013DF7D043EA46
:1007E0000603704794EA0C0F0CEA135518BF95EAFC
:1007F0000C0F0CD050EA410618BF52EA4306D1D183
:1008000081EA030101F000414FF0000070BD50EAA1
:10081000410606BF1046194652EA430619D094EA2B
:100820000C0F02D150EA013613D195EA0C0F05D115
:1008300052EA03361CBF104619460AD181EA030169
:1008400001F0004141F0FE4141F470014FF0000021
:1008500070BD41F0FE4141F4780170BD70B54FF0BC
:10086000FF0C4CF4E06C1CEA11541DBF1CEA13553C
:1008700094EA0C0F95EA0C0F00F0A7F8A4EB05041E
:1008800081EA030E52EA03354FEA013100F0888015
:100890004FEA03334FF0805545EA131343EA1263DE
:1008A0004FEA022245EA111545EA10654FEA002693
:1008B0000EF000419D4208BF964244F1FD0404F54C
:1008C000407402D25B084FEA3202B61A65EB0305A8
:1008D0005B084FEA32024FF480104FF4002CB6EB65
:1008E000020E75EB030E22BFB61A754640EA0C00E5
:1008F0005B084FEA3202B6EB020E75EB030E22BF25
:10090000B61A754640EA5C005B084FEA3202B6EB65
:10091000020E75EB030E22BFB61A754640EA9C0024
:100920005B084FEA3202B6EB020E75EB030E22BFF4
:10093000B61A754640EADC0055EA060E18D04FEAB2
:10094000051545EA16754FEA06164FEAC30343EA52
:1009500052734FEAC2025FEA1C1CC0D111F4801F1F
:100960000BD141EA00014FF000004FF0004CB6E718
:1009700011F4801F04BF01430020B4F1FD0C88BFB7
:10098000BCF5E06F3FF6AFAEB5EB030C04BFB6EBC2
:10099000020C5FEA500C50F1000041EB045170BDB5
:1009A0000EF0004E4EEA113114EB5C04C2BFD4EBE2
:1009B0000C0541EA045170BD41F480114FF0000E66
:1009C000013C90E645EA060E8DE60CEA135594EAE2
:1009D0000C0F08BF95EA0C0F3FF43BAF94EA0C0FE5
:1009E0000AD150EA01347FF434AF95EA0C0F7FF45A
:1009F00025AF104619462CE795EA0C0F06D152EAAE
:100A000003353FF4FDAE1046194622E750EA410691
:100A100018BF52EA43067FF4C5AE50EA41047FF4A2
:100A20000DAF52EA43057FF4EBAE12E74FF0FF3C07
:100A300006E000BF4FF0010C02E000BF4FF0010CD8
:100A40004DF804CD4FEA410C7FEA6C5C4FEA430C51
:100A500018BF7FEA6C5C1BD001B050EA410C0CBFA0
:100A600052EA430C91EA030F02BF90EA020F002002
:100A7000704710F1000F91EA030F58BF994208BF69
:100A800090422CBFD8176FEAE37040F00100704726
:100A90004FEA410C7FEA6C5C02D150EA013C07D17D
:100AA0004FEA430C7FEA6C5CD6D152EA033CD3D0C8
:100AB0005DF8040B704700BF8446104662468C46C2
:100AC0001946634600E000BF01B5FFF7B7FF0028F5
:100AD00048BF10F1000F01BD4DF808EDFFF7F4FF1E
:100AE0000CBF012000205DF808FB00BF4DF808EDA9
:100AF000FFF7EAFF34BF012000205DF808FB00BFCC
:100B00004DF808EDFFF7E0FF94BF012000205DF8ED
:100B100008FB00BF4DF808EDFFF7CEFF94BF0120A2
:100B200000205DF808FB00BF4DF808EDFFF7C4FF9B
:100B300034BF012000205DF808FB00BF4FEA410CE4
:100B40007FEA6C5C02D150EA013C0AD14FEA430CC7
:100B50007FEA6C5C02D152EA033C02D14FF0000004
:100B600070474FF0010070474FEA410212F5001242
:100B700015D211D56FF47873B3EB625212D94FEAE4
:100B8000C12343F0004343EA505311F0004F23FACE
:100B900002F018BF404270474FF00000704750EA23
:100BA000013005D111F0004008BF6FF000407047E0
:100BB0004FF00000704700BF4FEA4102B2F1E0433E
:100BC00024BFB3F5001CDCF1FE5C0DD901F0004C34
:100BD0004FEAC0024CEA5070B2F1004F40EB830084
:100BE00008BF20F00100704711F0804F21D113F1B0
:100BF0003872BCBF01F00040704741F480114FEAE9
:100C00005252C2F11802C2F1200C10FA0CF320FA71
:100C100002F018BF40F001004FEAC1234FEAD3238E
:100C200003FA0CFC40EA0C0023FA02F34FEA4303F8
:100C3000CCE77FEA625307D150EA01331EBF4FF081
:100C4000FE4040F44000704701F0004040F0FE409C
:100C500040F40000704700BF7BB972B90029BEBFE5
:100C600000204FF0004106E008BF00281CBF6FF0D5
:100C700000414FF0FF3000F0BDB9ADF1080C6DE957
:100C800004CE002909DB002B1ADB00F04DF8DDF85B
:100C900004E0DDE9022304B07047404261EB41010A
:100CA000002B1BDB00F040F8DDF804E0DDE9022357
:100CB00004B0404261EB4101524263EB4303704791
:100CC000524263EB430300F02FF8DDF804E0DDE966
:100CD000022304B0404261EB41017047524263EB92
:100CE000430300F021F8DDF804E0DDE9022304B05D
:100CF000524263EB4303704753B94AB9002908BF16
:100D000000281CBF4FF0FF314FF0FF3000F072B9E8
:100D1000ADF1080C6DE904CE00F006F8DDF804E052
:100D2000DDE9022304B070472DE9F047089E044630
:100D30008846002B4BD18A42154667D9B2FA82F217
:100D40004AB1C2F1200701FA02F320FA07F79540F1
:100D500047EA030894404FEA154E230CB8FBFEF710
:100D60001FFA85FC0EFB178843EA084307FB0CF1CA
:100D7000994209D9EB1807F1FF3080F01B819942A5
:100D800040F21881023F2B445B1AA4B2B3FBFEF081
:100D90000EFB103344EA034400FB0CFCA44509D9C4
:100DA0002C1900F1FF3380F00781A44540F2048143
:100DB00002382C4440EA0740A4EB0C0400271EB183
:100DC000D4400023C6E900433946BDE8F0878B4292
:100DD00009D9002E00F0EB800027C6E90001384653
:100DE0003946BDE8F087B3FA83F7002F47D18B422D
:100DF00002D3824200F2FA80841A61EB03030120DD
:100E00009846002EE0D0C6E90048DDE702B9FFDED3
:100E1000B2FA82F2002A40F08F80491B4FEA154E49
:100E20001FFA85F80127B1FBFEFC230C0EFB1C11F9
:100E300043EA014308FB0CF1994207D9EB180CF186
:100E4000FF3002D2994200F2CD808446591AA3B2F3
:100E5000B1FBFEF00EFB101443EA044408FB00F85B
:100E6000A04507D92C1900F1FF3302D2A04500F2AA
:100E7000B6801846A4EB080440EA0C409FE7C7F18F
:100E8000200CBB4022FA0CFE4EEA030E01FA07F4D6
:100E900020FA0CF521FA0CF34FEA1E482543B3FB68
:100EA000F8F92C0C08FB19331FFA8EFA44EA0343B5
:100EB00009FB0AF49C4202FA07F200FA07F10BD987
:100EC0001EEB030309F1FF3080F087809C4240F263
:100ED0008480A9F1020973441B1BADB2B3FBF8F087
:100EE00008FB103345EA034400FB0AFAA24508D97F
:100EF0001EEB040400F1FF336BD2A24569D902381E
:100F0000744440EA0940A0FB0289A4EB0A044C4562
:100F1000C2464B4654D351D0002E69D0B1EB0A05DE
:100F200064EB030404FA0CFCFD40FC404CEA0505AC
:100F3000C6E90054002747E7C2F1200320FA03F76F
:100F4000954001FA02F021FA03F34FEA154E3843B7
:100F5000010CB3FBFEF71FFA85F80EFB173341EACD
:100F6000034107FB08F38B4204FA02F407D969181E
:100F700007F1FF3C2FD28B422DD9023F2944CB1AD7
:100F800081B2B3FBFEF00EFB103341EA034100FBDC
:100F900008F38B4207D9691800F1FF3C17D28B4246
:100FA00015D902382944C91A40EA07473BE73746B2
:100FB000304609E70746E7E61846FBE64145ABD26F
:100FC000B8EB020A69EB0E0201381346A4E760464B
:100FD000E9E7184695E76746D1E781467CE702389E
:100FE0002C4447E7ACF1020C2B442FE7384608E7C6
:100FF0003746E9E6704700BF10B504460E4B187837
:101000004FF47A73B3FBF0F30C4A1068B0FBF3F0C3
:1010100000F06EFB68B90F2C01D901200AE0002214
:1010200021464FF0FF3000F0E9FA034B5C600020EE
:1010300000E0012010BD00BF0000002030000020B3
:1010400008B50B4B1A6842F400721A601A6842F431
:1010500080621A601A6842F480721A60032000F0FD
:10106000AFFA0020FFF7C8FF07F038F9002008BDED
:10107000003C0240034A1168034B1B780B44136089
:10108000704700BFE40A002000000020014B1868F0
:10109000704700BFE40A002038B50446FFF7F6FFAA
:1010A0000546B4F1FF3F02D0044B1B781C44FFF708
:1010B000EDFF401BA042FAD338BD00BF0000002066
:1010C00010B504464F4B5A6822F440325A605A68B1
:1010D00041680A435A600268536823F4807353607E
:1010E00002685368016943EA012353600268536848
:1010F00023F0407353600268536881680B43536068
:101100000268936823F40063936002689368C1687F
:101110000B439360826A3C4B9A425BD002689368AF
:1011200023F07063936002689368816A0B43936055
:101130000268936823F04053936002689368C16A21
:101140000B4393602268936823F002039360226844
:101150009368217E43EA4103936094F82030002B8A
:1011600049D0636A013B072B3FD82268536843F498
:10117000006353602268536823F46043536021681E
:101180004B68626A013A43EA42334B602268D36A91
:1011900023F47003D3622168CB6AE269013A43EA1F
:1011A0000253CB622268936823F400739360226831
:1011B000936894F8301043EA41239360226893685F
:1011C00023F48063936022689368616943EA812312
:1011D000936010BD0268936823F0706393600268A7
:1011E000936823F040539360ACE740F27571074871
:1011F00007F073F8B9E72268536823F4006353607B
:10120000C4E700BF002301400100000F18D400080C
:10121000002800F0E68010B504460268724B9A423E
:1012200004D040F24311714807F057F8636843B1A6
:10123000B3F5803F05D0B3F5003F02D0B3F5403F92
:1012400071D1A36843B1B3F1807F05D0B3F1007FC2
:1012500002D0B3F1407F6CD12369012B6FD8237E7C
:10126000012B72D8A36A7BB3B3F1807F2CD0B3F18A
:10127000007F29D0B3F1407F26D0B3F1806F23D017
:10128000B3F1A06F20D0B3F1C06F1DD0B3F1E06F08
:101290001AD0B3F1006F17D0B3F1106F14D0B3F1BF
:1012A000206F11D0B3F1306F0ED0B3F1406F0BD07F
:1012B000B3F1506F08D0B3F1606F05D0B3F1706F28
:1012C00002D04B4A934246D1E36813B1B3F5006FA5
:1012D00047D1E369013B0F2B49D894F83030012BFB
:1012E0004BD86369022B4ED894F82030012B50D88C
:1012F000A26A3F4B9A420AD0E36A43B1B3F1805FDE
:1013000005D0B3F1005F02D0B3F1405F47D1236C49
:10131000002B4AD0236C13F0100F4ED00120002375
:1013200084F83C3010BD4FF4A271304806F0D5FF70
:1013300087E740F245112D4806F0CFFF8CE74FF4C8
:10134000A3712A4806F0C9FF89E740F247112748F0
:1013500006F0C3FF86E74FF4A471244806F0BDFFF2
:10136000B2E740F24911214806F0B7FFB1E74FF468
:10137000A5711E4806F0B1FFAFE740F24B111B48C4
:1013800006F0ABFFADE74FF4A671184806F0A5FFD5
:10139000AAE740F24D11154806F09FFFA8E740F27A
:1013A0005111124806F099FFB1E7204606F0B2FF4E
:1013B0000023636484F83C30ACE7236C23F4885347
:1013C00023F0020343F0020323642046FFF778FE74
:1013D00000206064236C23F0030343F001032364C3
:1013E0009DE70120704700BF0020014018D400088D
:1013F0000100000F30B583B005460C460023019371
:101400000B68122B4ED86368013B0F2B50D8A36892
:10141000072B53D895F83C30012B00F0C7800123EF
:1014200085F83C302368092B4ED92868C2689BB2E6
:1014300003EB43031E3B072101FA03F322EA0303F4
:10144000C3602868C268A168238803EB43031E3B7E
:1014500001FA03F31343C3606368062B4AD8286874
:10146000426B03EB8303053B1F2101FA03F322EADE
:10147000030343632868426B636803EB8303053B04
:10148000218801FA03F3134343632A68484B9A42C5
:1014900060D02A68464B9A4265D0002085F83C000F
:1014A00003B030BD4FF4CB61424806F016FFAAE707
:1014B00040F259613F4806F010FFA8E740F25A6138
:1014C0003C4806F00AFFA5E7286802699BB203EBD7
:1014D0004303072101FA03F322EA030303612868A7
:1014E0000269A168238803EB430301FA03F3134362
:1014F0000361B1E70C2B16D82868026B03EB83035A
:10150000233B1F2101FA03F322EA03030363286844
:10151000026B636803EB8303233B218801FA03F327
:1015200013430363B1E72868C26A03EB8303413BBB
:101530001F2101FA03F322EA0303C3622868C26A87
:10154000636803EB8303413B218801FA03F31343F0
:10155000C3629AE72368122B9BD1174A536843F45E
:101560008003536095E72368103B012B95D8124AFE
:10157000536843F4000353602368102B8DD10F4B45
:101580001B6802F1467202F52E3202F28332A2FB90
:1015900003239B0C03EB83035A00019202E0019B9F
:1015A000013B0193019B002BF9D176E7022077E7FD
:1015B0000020014018D40008002301403000002022
:1015C00010B50446C31E042B0FD80A4AD36823F46F
:1015D000E0631B041B0C240204F4E064234343F087
:1015E000BF6343F40033D36010BD9221024806F07C
:1015F00074FEEAE700ED00E050D4000870B505463F
:101600000C4616460F2A25D80F2C28D81B4BDB6812
:10161000C3F30223C3F10702042A28BF0422191DC1
:10162000062921D9033B4FF0FF3101FA02F224EAE7
:1016300002049C4001FA03F326EA03063443002D1A
:1016400014DB2401E4B205F1604505F5614585F838
:10165000004370BDAA210A4806F03FFED4E7AB2143
:10166000074806F03AFED1E70023DCE705F00F0556
:101670002401E4B2034B5C55EBE700BF00ED00E052
:1016800050D4000814ED00E010B5041E0ADB002C55
:1016900007DB04F01F02640901239340044A42F867
:1016A000243010BDBE21034806F017FEEFE700BF4F
:1016B00000E100E050D4000810B5041E0FDB002C40
:1016C0000CDB04F01F026409012393402034064A16
:1016D00042F82430BFF34F8FBFF36F8F10BDCE2180
:1016E000024806F0FAFDEAE700E100E050D4000805
:1016F0000138B0F1807F0AD2064B5860064AF021CB
:1017000082F823100020986007221A607047012099
:10171000704700BF10E000E000ED00E00268D3B2C7
:10172000103B0B49A1FB03131B090A49C95CC165A6
:10173000032B06D822F47F7222F003028265806DAB
:10174000704722F47F7222F0030204328265F6E7CA
:10175000ABAAAAAAF8D30008836A826992B9012BBE
:101760000AD01BB1022B01D000207047C36A13F0CE
:10177000807F2CD100207047C36AB3F1C07F28D08E
:1017800000207047B2F5005F05D0022B29D9032B4A
:1017900015D000207047032B03D8DFE803F01C04AA
:1017A0001C0A00207047C36A13F0807F15D1002007
:1017B0007047C36AB3F1C07F11D000207047C36A7D
:1017C00013F0807F01D00120704700207047012076
:1017D00070470120704701207047012070470120A9
:1017E000704701207047000070B50446FFF74EFCBB
:1017F000002C00F03881054623689C4A934231D082
:10180000183293422ED0183293422BD01832934282
:1018100028D01832934225D01832934222D0183261
:1018200093421FD0183293421CD002F55672934255
:1018300018D01832934215D01832934212D0183271
:1018400093420FD0183293420CD01832934209D0F1
:101850001832934206D01832934203D0B8218448FC
:1018600006F03BFD6368A3B1B3F1007F11D0B3F183
:10187000806F0ED0B3F1C06F0BD0B3F1006F08D002
:10188000B3F1206F05D0B3F1406F02D0B3F1606FB8
:101890006DD1A3681BB1402B01D0802B6CD1E368C4
:1018A000B3F5007F01D0002B6BD12369B3F5806FB6
:1018B00001D0002B6AD163692BB1B3F5006F02D060
:1018C000B3F5805F67D1A3692BB1B3F5005F02D098
:1018D000B3F5804F64D1E36923B1B3F5807F01D0C4
:1018E000202B62D1236A43B1B3F5803F05D0B3F515
:1018F000003F02D0B3F5403F5CD1636A0BB1042BCB
:101900005DD1636AC3B1A36A032B5DD8E36A43B1B7
:10191000B3F5000F05D0B3F1807F02D0B3F1C07FE3
:1019200057D1236B43B1B3F5001F05D0B3F5800F3A
:1019300002D0B3F5C00F51D1002384F83430022314
:1019400084F835302268136823F00103136023689C
:101950001A6812F0010F46D0FFF798FB401B0528CC
:10196000F5D920236365032084F8350070BDB921C3
:101970003F4806F0B2FC8CE7BA213D4806F0ADFCCA
:101980008DE7BB213A4806F0A8FC8EE7BC21384819
:1019900006F0A3FC8FE7BD21354806F09EFC92E7D8
:1019A000BE21334806F099FC95E7BF21304806F088
:1019B00094FC97E7C0212E4806F08FFC9DE7C121DB
:1019C0002B4806F08AFC9CE7C621294806F085FCD6
:1019D0009CE7C721264806F080FCA2E7C8212448DE
:1019E00006F07BFCA8E71A68224810406168A268EC
:1019F0000A43E1680A4321690A4361690A43A1690C
:101A00000A43E1690A43216A0A430243616A0429DD
:101A10001ED01A602668756925F00705636A1D43A4
:101A2000042B07D1A36A1D43E36A1BB12046FFF7CD
:101A300093FE90B975612046FFF770FEE26D3F237B
:101A40009340836000206065012384F835308DE782
:101A5000E16A206B01430A43DBE740236365012011
:101A600084F8350082E7012080E700BF1060024063
:101A70008CD400083F8010F090F83530DBB2022B98
:101A800003D08023436501207047052380F835305B
:101A90000268136823F00103136000207047000000
:101AA000F0B583B0044600230193724B1D68724B5E
:101AB000A3FB0535AD0A876D3E68C26D08239340D0
:101AC000334210D003681A6812F0040F0BD01A6862
:101AD00022F004021A60C26D08239340BB60436D7C
:101AE00043F001034365E26D01239340334209D083
:101AF0002268526912F0800F04D0BB60636D43F01E
:101B000002036365E26D04239340334209D02268E7
:101B1000126812F0020F04D0BB60636D43F004033F
:101B20006365E26D10239340334224D0226812682B
:101B300012F0080F1FD0BB6023681A6812F4802FC0
:101B40000DD01B6813F4002F04D1236C9BB12046E9
:101B5000984710E0A36C73B1204698470BE01A68D1
:101B600012F4807F03D11A6822F008021A60236CF5
:101B70000BB120469847E26D20239340334255D065
:101B80002268126812F0100F50D0BB6094F8353004
:101B9000DBB2052B0ED023681A6812F4802F33D0E5
:101BA0001B6813F4002F2AD1636C002B3ED0204613
:101BB00098473BE02268136823F0160313602268FD
:101BC000536923F080035361236CA3B12268136827
:101BD00023F008031360E26D3F239340BB600023B2
:101BE00084F83430012384F83530236D002B3FD046
:101BF000204698473CE0A36C002BE7D1EBE7E36B72
:101C0000A3B12046984711E01A6812F4807F09D1E9
:101C10001A6822F010021A60002384F8343001237D
:101C200084F83530E36B0BB120469847636DFBB108
:101C3000636D13F0010F17D0052384F83530226847
:101C4000136823F001031360019B01330193AB423E
:101C500004D823681B6813F0010FF5D1002384F822
:101C60003430012384F83530E36C0BB120469847BB
:101C700003B0F0BD30000020B5814E1B274BDB6860
:101C800013F0100F07D0264AD36943F01003D36135
:101C9000224B1022DA60214BDB6813F0200F07D0B3
:101CA0001F4AD36943F00803D3611C4B2022DA603A
:101CB0001A4BDB6813F0400F07D0194AD36943F081
:101CC0000403D361154B4022DA60144BDB6813F038
:101CD000800F07D0124AD36943F00203D3610F4B40
:101CE0008022DA600D4BDB6813F4807F08D00C4A49
:101CF000D36943F00103D361084B4FF48072DA607B
:101D0000064BDB6813F0020F07D0054AD36943F096
:101D10002003D361014B0222DA607047003C02408D
:101D2000E80A002038B504460D4600F17843B3F5C3
:101D3000002F06D300F1604303F50843B3F5047F99
:101D40000CD2094B1A6922F440721A611A691A619D
:101D50001A6942F001021A61257038BD40F2BB21B8
:101D6000024806F0BAFAECE7003C0240C4D400088E
:101D700038B504460D4600F17843B3F5002F06D37D
:101D800000F1604303F50843B3F5047F0ED20A4B1C
:101D90001A6922F440721A611A6942F480721A6157
:101DA0001A6942F001021A61258038BD40F2A22171
:101DB000024806F092FAEAE7003C0240C4D4000868
:101DC00038B504460D4600F17843B3F5002F06D32D
:101DD00000F1604303F50843B3F5047F0ED20A4BCC
:101DE0001A6922F440721A611A6942F400721A6187
:101DF0001A6942F001021A61256038BD40F289215A
:101E0000024806F06AFAEAE7003C0240C4D400083F
:101E100070B5044616461D4600F17843B3F5002F11
:101E200006D300F1604303F50843B3F5047F11D2F4
:101E30000B4B1A6922F440721A611A6942F440721B
:101E40001A611A6942F001021A612660BFF36F8FAE
:101E5000656070BD40F26721024806F03EFAE7E790
:101E6000003C0240C4D40008094B1B69002B01DB75
:101E700000207047064B074A5A6002F188325A60C8
:101E80001B69002B01DB002070470120704700BF59
:101E9000003C02402301674538B50446154B00223B
:101EA000DA61FFF7F3F80546134BDB6813F4803F64
:101EB0000AD0B4F1FF3FF7D0CCB1FFF7E7F8401BF1
:101EC000A042F1D903200DE00B4BDB6813F0010FAA
:101ED00002D0094B0122DA60074BDB6813F4F97F6B
:101EE00001D1002038BDFFF7C9FE0120FAE7032029
:101EF000F8E700BFE80A0020003C0240F8B5214C9A
:101F0000247E012C3BD01F4616460D4604461D4B31
:101F100001221A7603281ED84CF25030FFF7BCFF7E
:101F2000014698B9E4B1012C1FD0022C22D03246D0
:101F30003B462846FFF76CFF4CF25030FFF7ACFFF2
:101F40000146114A136923F0010313610D4B00226E
:101F50001A760846F8BDA4210C4806F0BEF9DBE766
:101F6000F1B22846FFF7DEFEE6E7B1B22846FFF7FA
:101F7000FFFEE1E731462846FFF722FFDCE70221BA
:101F8000E7E700BFE80A0020003C0240C4D4000894
:101F900038B504460D46032816D8012D04D040F26A
:101FA000BD310C4806F099F90B4B1A6922F44072C6
:101FB0001A611A6942F004021A61186940EA0420A1
:101FC00040F48030186138BD4FF46F71014806F05D
:101FD00084F9E2E700D50008003C024038B5044629
:101FE0000D46072809D8032D0DD8ADB1012D2BD0F2
:101FF000022D0ED04FF440700FE040F2DB31144858
:1020000006F06BF9EFE74FF47771114806F065F9C8
:10201000EBE74FF4007000E000200E4B196921F44B
:10202000407119611A6902431A611A6922F0F802B3
:102030001A61186940EAC40040F0020018611A6988
:1020400042F480321A6138BD4FF48070E5E700BF7A
:1020500000D50008003C0240164B1B6813F4007FBB
:1020600010D0144B1A6822F400721A601A6842F4F5
:1020700000621A601A6822F400621A601A6842F458
:1020800000721A600B4B1B6813F4806F10D0094B61
:102090001A6822F480621A601A6842F480521A6048
:1020A0001A6822F480521A601A6842F480621A6038
:1020B000704700BF003C0240F8B52C4B1B7E012B43
:1020C00052D00E460446294B01221A7603689342E9
:1020D00029D84CF25030FFF7DFFE074600283ED1EA
:1020E0004FF0FF3333602368012B21D0E368A268EF
:1020F0001344013B072B2AD8A568E368A268134460
:10210000AB422AD9217C2846FFF768FF4CF25030B9
:10211000FFF7C2FE164A136923F0FA03136107465C
:10212000D0B90135E9E7AB21124806F0D6F8D0E77F
:102130006168207CFFF72CFF4CF25030FFF7ACFEBB
:1021400007460B4A136923F00403136105E0C3211A
:10215000084806F0C2F8CFE73560FFF77DFF034B74
:1021600000221A763846F8BD0227FBE7E80A00206D
:10217000003C024000D500082DE9F04383B08046C2
:102180000E46A24B984217D003F58063984213D0B5
:1021900003F5806398420FD003F5806398420BD01B
:1021A00003F58063984207D003F54063984203D05B
:1021B000B321974806F091F833689AB212B11B0C1C
:1021C0001B041BB1B421924806F087F87368012BF9
:1021D0001ED9112B1CD0022B1AD0122B18D08D4ACD
:1021E000934215D002F58012934211D002F580126D
:1021F00093420DD0A2F5F812934209D002F5801255
:10220000934205D002F58012934201D0032B04D1F2
:10221000B368022B06D8002445E0B5217C4806F0BF
:102220005CF8F5E7B6217A4806F057F8F3E7C821DD
:10223000774806F052F84AE0042300E000238B4080
:1022400003430232744941F82230744B1A68FB434D
:1022500003EA0201706810F4803F01D047EA0201EE
:102260006E4A1160526803EA0201706810F4003F80
:1022700001D047EA0201694A5160926803EA02010B
:10228000706810F4801F01D047EA0201634A916030
:10229000D2681340716811F4001F01D047EA0203AD
:1022A0005E4AD36001340F2C00F2AC800125A540BA
:1022B00037682F40BD42F5D173685A1E012A03D9F1
:1022C000112B01D0122B19D1F368032BAFD8D8F8FA
:1022D0000820610003238B4022EA0302F3688B404D
:1022E0001343C8F80830D8F8042022EA05027368BE
:1022F000C3F30015A5401543C8F80450D8F80C20C6
:102300004FEA4409032505FA09F5ED432A40B3686D
:1023100003FA09F31343C8F80C307368022B01D099
:10232000122B2BD13369CBB10C2B17D0012B15D02D
:10233000022B13D0042B11D0052B0FD0062B0DD060
:10234000072B0BD0082B09D00A2B07D0092B05D05F
:102350000F2B03D0E0212E4805F0BFFFE208083222
:1023600058F8220004F0070399000F238B4020EA5D
:10237000030033698B40034348F82230D8F800301B
:102380001D40736803F0030303FA09F31D43C8F803
:102390000050736813F0805F84D000230193204BBA
:1023A0005A6C42F480425A645B6C03F4804301939C
:1023B000019BA208911C184B53F8210004F0030361
:1023C00099000F238B4020EA0300104B98453FF4FF
:1023D00035AF03F5806398450ED003F580639845CB
:1023E0000CD003F5806398450AD003F580639845C7
:1023F0003FF422AF072322E7012320E702231EE751
:1024000003231CE703B0BDE8F08300BF00000240D7
:1024100040D500080000111000380140003C014088
:102420000038024038B505460C4621B12B691C42E4
:1024300007D1002038BD4FF4BF71034805F04DFFB0
:10244000F4E70120F6E700BF40D5000870B5064666
:1024500015460C4629B1012D09D875B92404B4617B
:1024600070BD40F29F11064805F037FFF3E74FF4C7
:10247000D071034805F031FFEFE7B461F0E700BF2A
:1024800040D5000838B505460C4629B16B6934EAD9
:10249000030307D0AC6138BD4FF4DB71034805F08E
:1024A0001CFFF3E72404AC61F5E700BF40D500084A
:1024B00003685A6912F4806F11D06FF480625A6118
:1024C00000230363202280F83D2080F83E30026C18
:1024D00042F00402026480F83C3001207047002082
:1024E0007047F8B506460C4617461D4622E0FEF733
:1024F000CDFD069BC01AA84200D8DDB90023336386
:10250000202286F83D2086F83E30326C42F02002D0
:10251000326486F83C3001201AE033685B6924EAB3
:1025200003039BB2B3FA83F35B099F420FD1B5F16A
:10253000FF3FDCD1C4F30743012BEED033689B6926
:1025400024EA03039BB2B3FA83F35B09EDE70020AF
:10255000F8BDF8B504460D4616461F463CE01A681D
:1025600042F400721A6023686FF480625A6100239B
:102570002363202284F83D2084F83E30226C42F010
:102580000402226484F83C30012033E0FEF77EFD33
:10259000C01BB04200D8FEB900232363202284F878
:1025A0003D2084F83E30226C42F02002226484F800
:1025B0003C3001201EE023685B6925EA03039BB2DF
:1025C000003318BF0123A3B123685A6912F4806F46
:1025D000C5D1B6F1FF3FD9D1C5F30743012BEAD0EE
:1025E00023689B6925EA03039BB2003318BF0123CC
:1025F000E9E70020F8BD0000F0B583B004460F46BF
:1026000015461E46C36A082B0DD0012B0BD013F5BF
:10261000803F08D0036B122B0AD10268136843F481
:102620008073136004E02268136843F480731360BE
:1026300000962B4600224FF001112046FFF751FF74
:1026400058B123681B6813F4807F2BD04FF40073BC
:1026500023640323184603B0F0BD2369B3F5804F0C
:102660000ED1236807F0FE071F6133462A460F4943
:102670002046FFF76EFF03460028EBD00123E9E771
:10268000FB11226803F0060343F0F00313613346A5
:102690002A4607492046FFF75CFF28B92368FFB2A6
:1026A0001F61E2E70323D5E70123D3E7020001001E
:1026B0000800010070B504460D46164623685B69A4
:1026C00013F0800F1CD12046FFF7F2FED0B9B5F110
:1026D000FF3FF3D0FEF7DAFC801BA84201D8002DA3
:1026E000ECD100232363202284F83D2084F83E307F
:1026F000226C42F02002226484F83C30012000E089
:10270000002070BD0120FCE72DE9F04184B00446B3
:10271000884616461F460B9D0268136843F4807373
:10272000136000950A9B00224FF00111FFF7D9FEBC
:1027300060B123681B6813F4807F4FD04FF400739F
:1027400023640323184604B0BDE8F081226808F032
:10275000FE0313612B460A9A21492046FFF7F9FE32
:1027600008B10123EEE70023039323685A6903921B
:102770009B690393039B2A460A992046FFF79AFF19
:10278000034658B1236C042B01D00123DAE72268F9
:10279000136843F4007313600123D3E7012F0ED0B5
:1027A0002368320A1A612A460A992046FFF782FFF7
:1027B000034678B1236C042B05D00123C2E72268BD
:1027C000F6B21661BEE72268136843F40073136023
:1027D0000123B7E72268F6B21661B3E70323B1E736
:1027E000020001002DE9F04184B004460E46174670
:1027F00098460B9D0268136843F480631360026877
:10280000136843F48073136000950A9B00224FF015
:102810000111FFF766FE68B123681B6813F4807F1F
:1028200000F089804FF4007323640323184604B03A
:10283000BDE8F081F6B2236806F0FE021A612B466D
:102840000A9A3F492046FFF784FE08B10123EDE7CD
:102850000023039323685A6903929B690393039BA4
:102860002A460A992046FFF725FF58B1236C042B0E
:1028700001D00123DAE72268136843F40073136080
:102880000123D3E7B8F1010F0DD12368FFB21F6117
:102890002A460A992046FFF70DFF20B3236C042B2C
:1028A0001AD00123C2E723683A0A1A612A460A9914
:1028B0002046FFF7FFFE58B1236C042B01D0012303
:1028C000B4E72268136843F4007313600123ADE793
:1028D0002368FFB21F61DBE72268136843F40073CB
:1028E00013600123A2E72268136843F48073136026
:1028F00000950A9B00224FF001112046FFF7F1FDE1
:1029000048B123681B6813F4807F16D04FF400731E
:10291000236403238AE7236846F001061E612B46E1
:102920000A9A07492046FFF714FE034600283FF4A1
:102930007DAF01237AE7032378E7032376E700BF1F
:102940000200010070B504460D46164623685B6917
:1029500013F0040F1CD12046FFF7AAFDD0B9B5F142
:10296000FF3FF3D0FEF792FB801BA84201D8002D59
:10297000ECD100232363202284F83D2084F83E30EC
:10298000226C42F02002226484F83C30012000E0F6
:10299000002070BD0120FCE770B505460C461646C8
:1029A0002B685A6912F0400F29D15A6912F0100FA2
:1029B00015D1FEF76BFB801BA04201D8002CEFD194
:1029C00000232B63202285F83D2085F83E302A6CB9
:1029D00042F020022A6485F83C30012070BD6FF07F
:1029E00010025A6100232B63202285F83D2085F8D0
:1029F0003E302A6C2A6485F83C300120EEE7002046
:102A0000ECE70000002800F03B81F8B504460368BD
:102A10009D4A93420CD002F58062934208D002F5A1
:102A20008062934204D040F2BD11984805F055FCF5
:102A30006368013B964A934200F2A580A3681BB1EC
:102A4000B3F5804F40F0A580E36823F47F7323F053
:102A50000303002B40F0A3802369B3F5804F03D01C
:102A6000B3F5404F40F0A1806369012B00F2A380D1
:102A7000A36933F0FE0340F0A480E36913B1402B57
:102A800040F0A580236A13B1802B40F0A68094F813
:102A90003D30002B00F0A780242384F83D302268CD
:102AA000136823F0010313602268136843F40043A2
:102AB00013602268136823F40043136001F028F8C0
:102AC0006268744B9A4200F29480734B98428CBFB8
:102AD00000230123002B40F0D580704BA3FB002383
:102AE0009B0C21684A6822F03F021A434A6025681D
:102AF0002A6A22F03F02666866498E427FD8013317
:102B000013432B622568E96921F44F4121F0FF014D
:102B10006368604A93427CD801385B00B0FBF3F3F2
:102B20000133C3F30B03042B38BF04230B43EB61C6
:102B300021680B6823F0C003E269206A0243134353
:102B40000B6021688B6823F4034323F0FF032269A1
:102B5000E068024313438B602168CB6823F0FF03D6
:102B60006269A06902431343CB602268136843F093
:102B70000103136000202064202384F83D3020638B
:102B800084F83E00F8BD4FF4DF71404805F0A5FB26
:102B900054E740F2BF113D4805F09FFB54E74FF466
:102BA000E0713A4805F099FB56E740F2C111374809
:102BB00005F093FB58E74FF4E171344805F08DFBC5
:102BC00056E740F2C311314805F087FB55E74FF453
:102BD000E2712E4805F081FB54E740F2C5112B4805
:102BE00005F07BFB53E784F83C30204605F0C6FB3C
:102BF00052E72B4B98428CBF002301236AE74FF426
:102C0000967101FB03F32749A1FB03139B090133D1
:102C100076E7A268BAB9461E03EB4307B6FBF7F6A0
:102C20000136C6F30B06B6FA86F6760936BBC2B98C
:102C3000013803EB4303B0FBF3F30133C3F30B029F
:102C400042F4004372E7461E03EB830707EB870756
:102C5000B6FBF7F60136C6F30B06B6FA86F676092A
:102C6000E4E7013803EB830303EB8303B0FBF3F2E8
:102C70000132C2F30B0242F4404357E7012355E708
:102C80000120704701207DE7005400407CD50008FA
:102C90007F1A0600A08601007F841E0083DE1B438E
:102CA000FF083D00D34D62102DE9F04184B0044689
:102CB0000E4690461F46FEF7E9F994F83D30DBB228
:102CC000202B04D00226304604B0BDE8F081054632
:102CD0000090192301224F492046FFF702FC0028EB
:102CE00040F0918094F83C30012B00F08E8001235D
:102CF00084F83C3023681A6812F0010F03D11A6877
:102D000042F001021A602268136823F40063136022
:102D1000212384F83D30102384F83E3000232364BF
:102D2000C4F824806785638D23853B4BE3622B4683
:102D30000A9A31462046FFF75FFC0646002866D116
:102D40000023039323685A6903929B690393039BAF
:102D500012E0236C042B01D00126B4E7226813682B
:102D600043F4007313600126ADE72A460A99204612
:102D7000FFF7E8FD00282CD1238D002B35D02A4603
:102D80000A992046FFF796FC0028E2D1626A236880
:102D900012781A61616A4B1C6362638D013B9BB2BE
:102DA0006385238D013B9BB223852268506910F017
:102DB000040FDAD0002BD8D04B781361636A01334B
:102DC0006362638D013B9BB26385238D013B238549
:102DD000CBE7236C042B01D0012674E7226813682B
:102DE00043F40073136001266DE72268136843F40F
:102DF00000731360202384F83D30002384F83E30B4
:102E000084F83C305FE702265DE702265BE7012697
:102E100059E700BF020010000000FFFF2DE9F0415C
:102E200082B004460F4690461E46FEF72FF905462F
:102E3000012E01D0102E09D194F83D30DBB2202BA9
:102E40000AD00223184602B0BDE8F08140F67311A3
:102E50004F4805F042FAEFE70095192301224D494A
:102E60002046FFF73EFB002840F08B8094F83C3072
:102E7000012B00F08880012384F83C3023681A6815
:102E800012F0010F03D11A6842F001021A602268A1
:102E9000136823F400631360212384F83D3040233A
:102EA00084F83E3000232364089B6362BDF824301D
:102EB0006385638D2385384BE36201950A9B0093FC
:102EC0003346424639462046FFF71EFC00285CD1B7
:102ED000238D002B34D02A460A992046FFF7EAFBBF
:102EE00010BB626A236812781A61616A4B1C6362C4
:102EF000238D013B9BB22385628D013A92B262859C
:102F00002268506910F0040FE2D0002BE0D04B781B
:102F10001361636A01336362238D013B2385638DF3
:102F2000013B9BB26385D3E7236C042B01D00123C3
:102F300088E72268136843F400731360012381E774
:102F40002A460A992046FFF7FDFC034658B1236C38
:102F5000042B01D0012375E72268136843F4007342
:102F6000136001236EE721680A6842F400720A6068
:102F7000202284F83D20002284F83E2084F83C2062
:102F800060E702235EE702235CE701235AE700BF04
:102F90007CD50008020010000000FFFF2DE9F04181
:102FA00086B004460F4690461E46FEF76FF805466B
:102FB000012E01D0102E09D194F83D30DBB2202B28
:102FC0000AD00226304606B0BDE8F08140F6EE1188
:102FD0009C4805F082F9EFE70095192301229A49F0
:102FE0002046FFF77EFA002840F03D8194F83C30FF
:102FF000012B00F03A81012384F83C3023681A68E1
:1030000012F0010F03D11A6842F001021A6022681F
:10301000136823F400631360222384F83D304023B7
:1030200084F83E30002323640C9B6362BDF8343087
:103030006385638D2385854BE36201950E9B009329
:103040003346424639462046FFF7CCFB0646002869
:1030500040F00D81238D5BB9029323685A69029277
:103060009A690292029A1A6842F400721A6072E037
:10307000012B0AD0022B1AD00023059323685A692A
:1030800005929B690593059B65E02268136823F40C
:10309000806313600023039323685A6903929A693B
:1030A0000392039A1A6842F400721A6053E022688D
:1030B000136823F4806313602268136843F4006389
:1030C00013600023049323685A6904929B69049354
:1030D000049B40E02A460E992046FFF75DFC00283D
:1030E00040F0C78023681A69636A1A70636A013303
:1030F0006362238D013B2385638D013B9BB2638516
:1031000029E000950E9B002251492046FFF7E9F97E
:10311000002840F0B0802268136843F40073136005
:1031200023681A69636A1A70626A531C6362238D8A
:10313000013B2385638D013B9BB2638523681B693B
:103140005370636A01336362238D013B2385638D72
:10315000013B9BB26385238D002B7BD0032B49D889
:10316000012BB7D0022BCCD000950E9B0022384902
:103170002046FFF7B6F900287FD12268136823F4B0
:103180008063136023681A69636A1A70636A013383
:103190006362238D013B2385638D013B9BB2638575
:1031A00000950E9B00222A492046FFF79AF9002835
:1031B00065D12268136843F40073136023681A69A9
:1031C000636A1A70626A531C6362238D013B238514
:1031D000638D013B9BB2638523681B695370636AEF
:1031E00001336362238D013B2385638D013B9BB2D9
:1031F0006385B0E72A460E992046FFF7CDFB0028ED
:103200003FD123681A69636A1A70626A531C636249
:10321000238D013B2385638D013B9BB2638523682E
:10322000596911F0040F96D01B695370636A01331A
:103230006362238D013B2385638D013B9BB26385D4
:1032400089E700BF7CD50008020010000000FFFFE6
:1032500004000100202384F83D30002384F83E3030
:1032600084F83C30AEE60226ACE60226AAE6012649
:10327000A8E60126A6E60126A4E60126A2E6012686
:10328000A0E601269EE600BF00283AD038B50446E5
:1032900002681D4B9A4203D09E211C4805F01DF880
:1032A0006368062B1ED8A368B3F5805F1FD223681E
:1032B0004CF6CC421A60236845F255521A602368D6
:1032C00062685A602368A2689A60FDF7DFFE0546CF
:1032D0002368DA6882B1FDF7D9FE401B3028F7D9A0
:1032E00003200DE09F21094804F0F7FFDBE7A02150
:1032F000064804F0F2FFDAE74AF6AA221A60002034
:1033000038BD0120704700BF00300040B4D5000830
:1033100003684AF6AA221A6000207047002800F0CD
:10332000648270B582B0044603680F2B39D82368D5
:1033300013F0010F4DD063682BB1B3F5803F02D07D
:10334000B3F5A02F32D1A54B9B6803F00C03042BDF
:1033500036D0A24B9B6803F00C03082B2BD063687C
:10336000B3F5803F5FD0B3F5A02F62D09B4B1A68B6
:1033700022F480321A601A6822F480221A6063688C
:10338000002B60D0FDF782FE0546944B1B6813F4BA
:10339000003F1ED1FDF77AFE401B6428F5D90320BB
:1033A00028E2E8218E4804F098FFC0E7ED218C4820
:1033B00004F093FFC7E7894B5B6813F4800FCED00E
:1033C000864B1B6813F4003F03D06368002B00F0AA
:1033D0000E82236813F0020F67D0E368012B41D8F7
:1033E00023691F2B44D87D4B9B6813F00C0F4AD0E8
:1033F0007A4B9B6803F00C03082B3FD0E368002B4B
:1034000077D0784B01221A60FDF740FE0546734BDA
:103410001B6813F0020F63D1FDF738FE401B022832
:10342000F5D90320E6E16D4A136843F48033136055
:10343000A5E76A4B1A6842F480221A601A6842F4BF
:1034400080321A609BE7FDF721FE0546634B1B683F
:1034500013F4003FBDD0FDF719FE401B6428F5D9D9
:103460000320C7E140F21F115D4804F036FFB7E7C3
:103470004FF490715A4804F030FFB4E7574B5B6843
:1034800013F4800FBAD1554B1B6813F0020F04D010
:10349000E368012B01D00120ACE1504A136823F00E
:1034A000F803216943EAC1031360236813F0080F8E
:1034B00049D06369012B2ED8636993B34A4B01222B
:1034C0001A60FDF7E3FD0546444B5B6F13F0020FF6
:1034D00039D1FDF7DBFD401B0228F5D9032089E136
:1034E0003E4A136823F0F803216943EAC1031360DD
:1034F000DBE73C4B00221A60FDF7C8FD0546374B61
:103500001B6813F0020FD0D0FDF7C0FD401B02284E
:10351000F5D903206EE14FF4B071314804F0DDFEBF
:10352000CAE7314B00221A60FDF7B0FD05462B4B70
:103530005B6F13F0020F06D0FDF7A8FD401B0228B9
:10354000F5D9032056E1236813F0040F00F08780BB
:10355000A368012B01D9052B38D1204B1B6C13F02C
:10356000805F39D1002301931C4B1A6C42F08052CA
:103570001A641B6C03F080530193019B01251B4BC4
:103580001B6813F4807F33D0A368012B44D0052B34
:1035900048D0124B1A6F22F001021A671A6F22F0FC
:1035A00004021A67A368002B46D0FDF76FFD06469C
:1035B0000A4B1B6F13F0020F4FD1FDF767FD801B05
:1035C00041F288339842F3D9032013E14FF4C671D6
:1035D000034804F082FEC0E70025D0E7003802402F
:1035E000F0D5000800004742800E474200700040BE
:1035F000834A136843F480731360FDF747FD064662
:103600007F4B1B6813F4807FBED1FDF73FFD801B0D
:103610000228F5D90320EDE07A4A136F43F0010345
:103620001367BFE7774B1A6F42F004021A671A6FED
:1036300042F001021A67B5E7FDF728FD0646714B17
:103640001B6F13F0020F08D0FDF720FD801B41F225
:1036500088339842F3D90320CCE0002D3BD1A369F5
:10366000022B3ED8A369002B00F0C380654A926804
:1036700002F00C02082A00F09080022B79D1E36955
:1036800013B1B3F5800F32D1236A3F2B35D8636A6B
:10369000323BB3F5BF7F36D8A36A022B05D0042B8B
:1036A00003D0062B01D0082B33D1E36A023B0D2B4C
:1036B00035D8554B00221A60FDF7E8FC0546514B02
:1036C0001B6813F0007F30D0FDF7E0FC401B0228A0
:1036D000F5D903208EE04B4A136C23F0805313641A
:1036E000BDE740F2CF11494804F0F7FDBAE74FF4C7
:1036F000EC71464804F0F1FDC6E740F2D9114348A9
:1037000004F0EBFDC3E74FF4ED71404804F0E5FD34
:10371000C2E740F2DB113D4804F0DFFDC5E74FF49E
:10372000EE713A4804F0D9FDC3E7E369226A134316
:10373000626A43EA8213A26A5208013A43EA0243E8
:10374000E26A43EA02632F4A53602F4B01221A6058
:10375000FDF79CFC04462B4B1B6813F0007F06D141
:10376000FDF794FC001B0228F5D9032042E000205D
:1037700040E0254B00221A60FDF788FC0446214BEF
:103780001B6813F0007F06D0FDF780FC001B0228A9
:10379000F5D903202EE000202CE0012B2CD0194B72
:1037A0005B6803F48001E269914201D0012021E0CD
:1037B00003F03F02216A8A4201D001201AE0616AC7
:1037C00047F6C0721A408A4201D0012012E003F489
:1037D0004032A16A8A4201D001200BE003F07063FD
:1037E000E26A93420AD0012004E0012070470120E0
:1037F00000E0002002B070BD0120FBE70020F9E7E7
:10380000007000400038024060004742F0D50008D8
:10381000324B9B6803F00C03042B5CD0082B01D0C7
:103820002F4870472DE9F04B2C4B5A6802F03F02AD
:103830005B6813F4800F2BD0284B5B68C3F38813AD
:103840001E4600275C010025E41A65EB0705A90167
:1038500041EA9461A001001B61EB0501CB0043EA42
:103860005073C400A01943EB07014B0243EAD05345
:103870004402204619460023FDF73EFA174B5B68C9
:10388000C3F3014301335B00B0FBF3F0BDE8F08B01
:10389000124B5B68C3F388131E4600275C010025AA
:1038A000E41A65EB0705A90141EA9461A001001B38
:1038B00061EB0501CB0043EA5073C400A01943EB50
:1038C00007018B0243EA90538402204619460023E5
:1038D000FDF712FAD2E70348704700BF00380240F4
:1038E0000024F40000127A00002800F0FA8070B57D
:1038F00004460D460368013B0E2B11D8072D15D841
:103900007A4B1B6803F00F03AB4215D2EBB2774A38
:103910001370136803F00F03AB420DD0012070BD8C
:1039200040F25121724804F0D8FCE7E740F25221FE
:103930006F4804F0D2FCE3E7236813F0020F29D0AC
:1039400013F0040F04D06B4A936843F4E053936080
:10395000236813F0080F04D0664A936843F4604369
:103960009360A3687BB1802B0DD0902B0BD0A02B44
:1039700009D0B02B07D0C02B05D0D02B03D0E02B23
:1039800001D0F02B33D15B4A936823F0F003A16898
:103990000B439360236813F0010F42D06368032B3D
:1039A0002BD86368012B2ED09A1E012A32D9514A96
:1039B000126812F0020F00F096804E498A6822F0D9
:1039C000030213438B60FDF761FB0646494B9B687E
:1039D00003F00C036268B3EB820F22D0FDF756FBB5
:1039E000801B41F288339842F0D9032097E740F2D8
:1039F00075213F4804F071FCC5E74FF41F713C4846
:103A000004F06BFCCDE73B4A126812F4003FD4D1BE
:103A1000012084E7374A126812F0007FCDD10120DF
:103A20007DE7324B1B6803F00F03AB4209D9EAB2C2
:103A30002E4B1A701B6803F00F03AB4201D001201C
:103A40006DE7236813F0040F14D0E3685BB1B3F59E
:103A5000805F08D0B3F5A05F05D0B3F5C05F02D09A
:103A6000B3F5E05F31D1234A936823F4E053E16872
:103A70000B439360236813F0080F15D023695BB1E3
:103A8000B3F5805F08D0B3F5A05F05D0B3F5C05F94
:103A900002D0B3F5E05F1ED1164A936823F4604369
:103AA000216943EAC1039360FFF7B2FE114B9B68A3
:103AB000C3F30313104AD35CD840104B1860104B6B
:103AC0001868FDF799FA002029E740F2BA21084862
:103AD00004F003FCC7E740F2C121054804F0FDFBF8
:103AE000DAE701207047012019E700BF003C0240DF
:103AF000F0D500080038024000D400083000002053
:103B000004000020014B1868704700BF30000020FF
:103B100008B5FFF7F7FF044B9B68C3F38223034A02
:103B2000D35CD84008BD00BF0038024010D4000864
:103B300008B5FFF7E7FF044B9B68C3F34233034A22
:103B4000D35CD84008BD00BF0038024010D4000844
:103B5000F8B505460F4616461C462B689B6837EAA3
:103B600003030CBF01230023B34237D0B4F1FF3F5E
:103B7000F3D0FDF78BFA069BC01AA04201D2002CAD
:103B8000EBD12A68536823F0E00353606B68B3F508
:103B9000827F0BD0AB6AB3F5005F14D0012385F8A8
:103BA0005130002385F85030032018E0AB68B3F59E
:103BB000004F02D0B3F5806FECD12A68136823F070
:103BC00040031360E6E72A68136823F40053136088
:103BD0002A68136843F400531360DFE70020F8BD40
:103BE00030B585B0164C2468164DA5FB0434640D21
:103BF0004FF47A7505FB04F403944468B4F5827FAE
:103C00000BD0039BC3B1039B013B039303689B68E9
:103C100013F0800FF5D100230FE00B46044600920D
:103C200000228021FFF794FF034630B1636D43F01B
:103C300020036365032300E00023184605B030BD70
:103C400030000020819F5E16002800F0C48010B56F
:103C500004460368614A934210D0A2F57842934229
:103C60000CD002F58062934208D002F5784293426C
:103C700004D04FF4A1715A4804F02FFB636813B1CC
:103C8000B3F5827F6BD1A3682BB1B3F5806F02D0FF
:103C9000B3F5004F69D1E368B3F5006F01D0002B95
:103CA00069D1A369B3F5007F03D013B1B3F5802FB9
:103CB00067D1E3696BB1082B0BD0102B09D0182BFF
:103CC00007D0202B05D0282B03D0302B01D0382B48
:103CD0005DD1236A0BB1802B5FD1636A0BB1102BCE
:103CE00061D1636A33B923690BB1022B61D1636976
:103CF000012B64D80023A36294F85130002B64D0C8
:103D0000022384F851302268136823F040031360C3
:103D10006368A2681343E26813432269134362692C
:103D20001343A26902F400721343E2691343226A47
:103D30001343A16A22680B431360638B03F00403EF
:103D4000616A22680B4353602268D36923F40063DD
:103D5000D36100206065012384F8513010BD40F22A
:103D600043111F4804F0B9FA8DE74FF4A2711C48C3
:103D700004F0B3FA8FE740F24511194804F0ADFAA8
:103D80008FE74FF4A371164804F0A7FA91E740F2C9
:103D90004711134804F0A1FA9BE74FF4A4711048AF
:103DA00004F09BFA99E740F249110D4804F095FAA6
:103DB00097E74FF4A6710A4804F08FFA97E740F2AC
:103DC0004D11074804F089FA94E784F850302046F2
:103DD00004F00EFB94E70120704700BF0030014063
:103DE00028D600082DE9F04182B0044688461746DF
:103DF0001D46836813B1B3F5004F19D194F85030C4
:103E0000012B00F0C580012384F85030FDF73EF906
:103E1000064694F85130DBB2012B0FD0022001236B
:103E200084F85130002384F8503002B0BDE8F081AE
:103E300040F2F221574804F050FADFE7B8F1000FE2
:103E400000F09880002F00F09780032384F8513011
:103E500000236365C4F83080A786E786A363A38741
:103E6000E38763642364A368B3F5004F1CD0236821
